:020000040000FA
:02000000050AEF
:06000A00A304C304A404DA
:10001000C404E404000C0200000C2500000C2600BF
:10002000000C2700000C2800000C2900060C05001D
:10003000000C0600000C0700000C0800000C090072
:10004000A404C404E40405047300F4046A006C000E
:100050006D00010C2E0030007100010C37003800DB
:100060003404140C3200010C2F00A404C405E40471
:10007000230C3100020C32002C0C3300050C340030
:10008000A404C404E4047404B404A405C404E4048F
:1000900011053104F104A404C404E4040A0C36007C
:1000A000A404C405E404050C3700050C3800100452
:1000B0005004190C35000000A405C404E404070C26
:1000C0003200330034003500F00C36003700320CBB
:1000D0003800B00490047004500410043004A404E8
:1000E000C404E4045404A404C405E4047004A40493
:1000F000C404E4047B0AA404C404E4040504A404C2
:10010000C404E404700C39004507C70AF902840AE4
:100110004506880A0A0C3600F407910A0505040C06
:100120000500140C2400500C39004506C70AF902DA
:10013000950A060C39004506C70AF9029B0AE40035
:10014000080C3900F406B00A4507A40A2506030581
:10015000250703046003F902A40AF602990AC10AFA
:10016000600303062505030725044507B50AF902C0
:10017000B00A6003F602990A060C05000504F404AF
:10018000D304280C39004506CA0AF902C30A05043B
:100190000B057B0AA404C405E404A404C405E40418
:1001A00018028A004306DD0A0A023800F702DD0A57
:1001B000070C3700010CB001DD0AA404C404E404F8
:1001C0007407F20AA404C405E40412028D00430774
:1001D000F20A11028C004307F20A8905F004B00705
:1001E000F005F80AA404C405E4048904F004B0048A
:1001F000A404C404E404B4070D0BA404C405E4047B
:1002000014028D0043070D0B13028C0043070D0BE6
:10021000A905D0049007D005130BA404C405E40479
:10022000A904D00490040000A404C405E404F0066A
:100230001B0BD0075B0BA405C404E4041107360BA9
:100240007900020C3B006504200C3A00FA02260BF0
:100250006505200C3A00FA022B0BF902230BFB0276
:10026000230B020C3B00110431055B0B000031072E
:10027000500B7900020C3B006504210C3A00FA0295
:100280003F0B6505210C3A00FA02440BF9023C0BC6
:10029000FB023C0B020C3B003104F105D0045B0B6C
:1002A0000000F1075A0BF8025B0B320C3800110505
:0E02B0003104F10400000000A305C304000A9D
:10040000A405C404E404C00C0800060A070A100688
:100410000D0AC8061F0AF2021F0A1005C8071A0AA9
:10042000F3021F0A5005070C32003300F00C3600AF
:1004300010041F0AF6021F0A9005F00C3600300661
:10044000250AE806370AF402370A3005E807320AB7
:10045000F502370A7005070C34003500F00C370040
:100460003004370AF702370AB005F00C3700000CE9
:1004700008009006460A50064C0A9006460AB00646
:10048000490A70068F0AB006490AE90AB007720ADB
:10049000CF0A9007A40ACF0AA404C404E4043406D3
:1004A0005D0A03047703B707570A010C3700000001
:1004B000A405C404E40450043F0AA404C404E404EE
:1004C000030478033706660A5707680A98066A0A1B
:1004D000D8076C0A010C38000000A405C404E40429
:1004E00050043F0AA405C404E4045007820A5004DF
:1004F0009004A404C404E404040CB401A405C404DA
:10050000E4043F0AA404C404E40454063404540775
:100510003405010C3800A405C404E4043F0AA40413
:10052000C404E40434079A0AD405A405C404E4040A
:100530007004E90AA404C405E404B0059005A40508
:10054000C404E4047004E90AA405C404E4047007C4
:10055000BA0A7004B004A404C404E4043406E90A2A
:10056000A404C405E404080CB0019405A405C40463
:10057000E404E90AA404C404E4043407C40A370602
:1005800074045706B404E90AA404C405E40470061C
:10059000500470075005A405C404E404E90AA40546
:1005A000C404E404F3057004700450047004A4044B
:1005B000C404E404F305F4056A006C00140C2D0077
:1005C00077001705000C0800A404C405E4045004D7
:0A05D00030040000C305A304800AF4
:10080000A404C404E4047A0039000A0C9900030724
:100810000C0A3900FA03050A9A03F9010008A40436
:10082000C404E4043407200AA404C405E404300723
:10083000200AA404C404E4041905390559057905FE
:10084000A404C404E4040008A404C404E4043407B5
:10085000350AA404C405E4043007350AA404C4041A
:10086000E4049905B905D905F905A404C404E40410
:10087000000818060F0938062409000858060F0951
:1008800078062409000898060F09B806240900080C
:10089000A404C405E40439000C0C3A00C904500750
:1008A0006A0A1A02990003075F0A0C0C99003600C5
:1008B000360243075D0A0C0C3600C9056C0AA40415
:1008C000C405E4041902360036024307690A0C0C19
:0A08D00036006C0A19023600000819
:10090000A404C404E404000C08001707A80AA40403
:10091000C404E4040A0200093909190226000C0281
:1009200000093E09190227000D024809A404C40564
:10093000E4041602A404C404E404000943091902EF
:1009400028006505E9047406E905B406E905140BF9
:100950003707CC0AF10C2600A404C405E4041102F4
:10096000A404C404E4040009390919022700A404FA
:10097000C405E40412024809A404C405E4041602F0
:10098000A404C404E40400093E0919022800650512
:10099000E9047406E905140B5707F00AF20C260067
:1009A000A404C405E4041302A404C404E404000978
:1009B000390919022700A404C405E40414024809F3
:1009C000A404C405E4041602A404C404E404000955
:1009D0003E09190228006505E904B406E905140B6F
:1009E00077070C0BA404C404E404C9041102000931
:1009F000390919022600100200093E0919022700D0
:100A00000E0200094309190228006504E90474066E
:100A1000E905B406E905140B9707870AA404C40581
:0E0A2000E4041007870AF20AC305A305000AC2
:100C0000A404C404E4043407390B17060E0A37069B
:100C10004B0A5706960A7706E10A390BA404C40466
:100C2000E404D407390B1807160AD3053807190A44
:100C3000D3055807210AAC0203043C0C8C000306C0
:100C40006C0078072A0A0A0CEC0103043C0C8C00A7
:100C500003062C009807320AAD020304180C8D001D
:100C600003066D00B807450A0A0CED010304180CD1
:100C70008D000307440A03041E0C8D000307420A7B
:100C80002D00440A140CAD000000A404C404E404C4
:100C9000F405D404390BA404C404E404D407390BC8
:100CA00018075B0AA404C405E404B10203043C0C65
:100CB000910003067100A404C404E40438076A0A1E
:100CC000A404C405E4040A0CF10103043C0C9100E3
:100CD00003063100A404C404E4045807780AA404F9
:100CE000C405E404B2020304180C92000306720067
:100CF000A404C404E4047807900AA404C405E4042A
:100D00000A0CF2010304180C92000307900A030472
:100D10001E0C920003078E0A3200900A140CB200D7
:100D2000A404C404E404D4047405390BA404C40466
:100D3000E404D407390B1807A60AA404C405E40484
:100D4000B30203043C0C930003067300A404C40420
:100D5000E4043807B50AA404C405E4040A0CF3014A
:100D600003043C0C930003063300A404C404E4040D
:100D70005807C30AA404C405E404B4020304180C0D
:100D8000940003067400A404C404E4047807DB0A96
:100D9000A404C405E4040A0CF4010304180C940030
:100DA0000307DB0A03041E0C94000307D90A34006E
:100DB000DB0A140CB400A404C404E404D404B40591
:100DC000390BA404C404E404D407390B1807EF0A50
:100DD000B1020304460C910003067100310B380781
:100DE000F90A0A0CF1010304460C91000306710094
:100DF000310B5807030BB00203040D0C90000307DE
:100E0000030B010C30007807150B0A0CF0010304EA
:100E10000D0C90000307150B0304140C900003073E
:100E2000130B3000150B0A0CB00098071F0BAE0215
:100E30000304200C8E0003071F0B010C2E00B807C3
:100E4000310B0A0CEE010304200C8E000307310B5A
:100E50000304280C8E0003072F0B2E00310B1E0CF1
:100E6000AE00A404C404E404F405D4043002430630
:100E7000B0020000A404C405E404F502440B190CFC
:100E80003500020CB001440BA404C404E404A30420
:040E9000C3047F0A0E
:021FFE00F90FD9
:00000001FF
